:020000040000FA
:1000000007309F000030831600309F008600850077
:10001000831231200E20192025200D283030840035
:100020001030A30023085A208000840AA30B122852
:10003000080080303A200830A2003F3084000008D9
:1000400046208403A20B1F280800C0303A20083045
:10005000A20037308400000846208403A20B2B281E
:10006000080038303A2001303A2003303A200F306F
:100070003A200800860052200430850052200030CB
:10008000850052200430850052200800860052204E
:10009000063085005220023085005220063085004F
:1000A000522008006430A100A000A00B5528A10B2D
:1000B0005428080082072034203445344434553411
:1000C00050344934433420342034313436344634C7
:0800D000363432343834203498
:02400E00293F48
:00000001FF
